:020000040000FA
:100000008316003085008312831601308600831228
:100010000030850000309600053C9700970A0000EC
:10002000063086000A309A000A3099000A3098009B
:10003000E620003086000A309A000A3099000A3023
:100040009800E620960A970B0F28861489308C00BA
:10005000B2308D000C308E0000308F0000309000E8
:10006000003091000618322807309600003C9E00B0
:100070009E099E0A9E0A0000003092000030930004
:10008000DD20920A1208643C031847282C2800003F
:10009000061C4028DD20930A1308FA3C0318512857
:1000A0002C28000006184A281208130203185A28A0
:1000B00003145C280000031000008F0D96039E0BB4
:1000C0003B2807309600003CA000A009A00AA00A27
:1000D00000000030920000309300DD20920A1208E8
:1000E000643C031874282C280000061C6D28DD20B1
:1000F000930A1308FA3C03187E282C2800000618DF
:10010000772812081302031887280314892800008F
:1001100003100000900D9603A00B6828073096008E
:10012000003CA100A109A10AA10A00000030920030
:1001300000309300DD20920A1208643C0318A128C5
:100140002C280000061C9A28DD20930A1308FA3C8C
:100150000318AB282C2800000618A4281208130244
:100160000318B4280314B628000003100000910DF2
:100170009603A10B95280F080C020319C0282C2800
:10018000000010080D020319C6282C2800001108D1
:100190000E020319CD282C28DB2800008610061536
:1001A000851464309A000A3099000A309800E620DD
:1001B00086140611851000002C281C309400013094
:1001C0009500950BE128940BDF28080018089B0088
:1001D00019089C00F9309D0000009D0BEC289C0B39
:0E01E000EA289B0BE8289A0BE628080000008E
:02400E00FB3F76
:00000001FF
